:020000040800F2
:1000000000070020F101000809240008C1230008AE
:10001000E9230008C1230008E1230008F3010008D8
:10002000F3010008F3010008F3010008FD330008A4
:10003000F3010008F3010008F3010008F3010008D0
:10004000F3010008F3010008F3010008F3010008C0
:10005000F3010008F3010008CD410008F541000854
:100060001D420008454200086D420008F3010008E7
:10007000F3010008F3010008F3010008F301000890
:10008000F3010008F3010008F301000875230008DC
:10009000A1230008B1230008F301000895420008DD
:1000A000F3010008F3010008F3010008F301000860
:1000B00091430008F3010008F3010008F301000870
:1000C000F3010008F3010008F3010008F301000840
:1000D000F3010008694300087D430008F3010008AC
:1000E000F9420008F3010008F3010008F3010008D9
:1000F000F3010008F3010008F3010008F301000810
:10010000F3010008F3010008F3010008F3010008FF
:10011000F3010008F3010008F3010008F3010008EF
:10012000F3010008F3010008F3010008F3010008DF
:10013000F3010008F3010008F3010008F3010008CF
:10014000F3010008F3010008F3010008F3010008BF
:10015000F3010008F3010008F3010008F3010008AF
:10016000F3010008F3010008F3010008F30100089F
:10017000F3010008F3010008F3010008F30100088F
:10018000F3010008F3010008F3010008F30100087F
:10019000F3010008F3010008F3010008F30100086F
:1001A000F3010008F3010008F3010008F30100085F
:1001B000F3010008F3010008F3010008F30100084F
:1001C000F3010008F3010008F3010008F30100083F
:1001D000F3010008F3010008F3010008F30100082F
:1001E000C50F000800000000000000000000000033
:1001F00002E000F000F8FEE772B6374880F30888A6
:10020000364880F3098836483649086040F20000D5
:10021000CCF200004EF63471CEF200010860BFF35C
:100220004F8FBFF36F8F40F20000C0F2F0004EF628
:100230008851CEF200010860BFF34F8FBFF36F8F7C
:100240004FF00000E1EE100A4EF63C71CEF20001D4
:100250000860062080F31488BFF36F8F03F0C0FDA1
:1002600003F052FE4FF055301F491B4A91423CBFEC
:1002700041F8040BFAE71D49184A91423CBF41F886
:10028000040BFAE71A491B4A1B4B9A423EBF51F82E
:10029000040B42F8040BF8E700201849184A914271
:1002A0003CBF41F8040BFAE703F09EFD03F07AFE31
:1002B000144C154DAC4203DA54F8041B8847F9E797
:1002C00000F042F8114C124DAC4203DA54F8041B12
:1002D0008847F9E703F086BD0007002000230020CF
:1002E0000000000808ED00E00001002000070020E9
:1002F000C04C000800230020802300208023002021
:1003000028520020E0010008E4010008E401000890
:10031000E40100082DE9F04F2DED108AC1F80CD052
:10032000C3689D46BDEC108ABDE8F08F002383F3BF
:1003300011882846A047002003F0BCF9FEE703F02F
:1003400045F900DFFEE70000F8B500F04DFE03F0D0
:10035000E1FC074603F030FD064600283DD12B4B5B
:100360009F423AD001339F423AD0294B27F0FF02F7
:100370009A4238D1F8B200F043FC354642F210748C
:1003800000F044FC08B10024254601F019F970B3CF
:10039000032000F043F80024254636B11D4B9F4250
:1003A00003D003F001FD00242546002003F0BCFC2F
:1003B000194B1B691B071FD40DB100F045F800F065
:1003C00091FC02F029F80546C4B102F025F8401B63
:1003D000A04213D900F038F8F3E735460024CFE700
:1003E00004460125CCE705464FF47A74C8E7B4F516
:1003F0007A7F08BF0125D0E70024E0E700F0BAFCCF
:100400004FF47A7003F05CF9DEE700BF010007B03B
:10041000000008B0263A09B000040240084B1870EA
:1004200003280CD8DFE800F008050208022000F0DD
:1004300039BE022000F02CBE024B00225A607047E9
:10044000802300208423002010B501F0B9F830B1DA
:10045000204B03221A70204B00225A6010BD1F4B04
:100460001F4A1C4619680131F8D004339342F9D170
:1004700062681C4B9A42F1D91B4B9B6803F10063E5
:1004800003F580339A42E9D203F062FC03F074FC76
:10049000002000F0C3FD0220FFF7C0FF134B1A6CD1
:1004A00000221A64196E1A66196E596C5A64596ED4
:1004B0005A665B6E72B64FF0E0233021C3F8084DE8
:1004C000D4E9003281F311889D4683F308881047F0
:1004D000C4E700BF8023002084230020000001081F
:1004E00020000108FFFF0008002300200038024020
:1004F000094A136849F2690099B21B0C00FB0133E9
:100500001360064B186844F2506182B2000C01FB84
:100510000200186080B270471823002014230020C6
:1005200010B500211022044600F0D8FD034B03CB88
:10053000206061601868A06010BD00BF107AFF1FC6
:100540002DE9F041ADF54E7D0DF134086CAC40F273
:10055000751207460D460EA80021C8F8001000F0DD
:10056000BDFD4FF4C4720021204600F0B7FD01F03C
:1005700053FF274B4FF47A72B0FBF2F0186093E808
:100580000700022384E807000DF5E9702382FFF7D6
:10059000C7FF4EF603131F49238407A804F09CFAF3
:1005A000162384F832310DF2E32207AB0DF12C0C47
:1005B0001E4603CE664510605160334602F10802C4
:1005C000F6D130681060B3889380414601222046FE
:1005D00000F0D0FD00230393AB7E029305F11903D5
:1005E000019380B20123CDE904800093E97E06A344
:1005F000D3E90023384602F0D7FA0DF54E7DBDE869
:10060000F08100BFAFF300809E6AC421818A46EE6C
:100610008C230020E84A00082DE9F0412C4C237A75
:10062000DAB080460D465BBB27A9284600F0B2FE33
:100630000746002842D19DF89D60C82E3ED801464D
:100640004FF4A662204600F049FD4FF48073C4F8D1
:10065000F8314FF40073C4F80C334FF44073C4F80E
:10066000203432460DF19E0104F1090000F024FD12
:1006700026449DF89C30777223720BB9EB7E23726F
:100680008122002106AC27A800F028FD0122214686
:1006900027A800F0BBFE00230393AB7E029305F175
:1006A000190380B201932823CDE904400093E97E29
:1006B00005A3D3E90023404602F076FA5AB0BDE81C
:1006C000F08100BFAFF3008026417272DF25D7B7FB
:1006D000B0440020F0B5254E4FF48A7505FB006547
:1006E000F1B096F8D83085F8DC300024D8222146C5
:1006F00085F8E8403AA800F0F1FC06F1090000F0A6
:10070000E5FCD5F8E4308DF8F000C2B206AF06F192
:1007100009010DF1F100CDE93A3400F0CDFC394684
:1007200001223AA800F09EFE80B2CDE904700823B1
:100730000127CDE9023706F1D80301933023009356
:10074000317A0B4807A3D3E9002302F02DFAA04227
:1007500006DD01F061FEC5F8E000384671B0F0BD7D
:100760002046FBE778F6339F93CACD8DB044002036
:10077000A43300202DE9F0411D4D1E4E1E4F86B0C2
:10078000284602F03DFA034658B30024CDE903445D
:10079000ADF81440027B8DF81420996840680294EB
:1007A00003AA03C21B68DFF8548043F0004302939E
:1007B00001F034FE821941F10003009402A9384689
:1007C00001F0DCF8A04205DD284602F01DFA88F8A9
:1007D0000040D5E798F80030072B05D8013388F89A
:1007E000003006B0BDE8F081014802F00DFAF8E7EC
:1007F000A433002040420F00D8330020E5490020F8
:1008000070B50D4614461E4602F02AF950B9022E64
:1008100010D1012C0ED112A3D3E90023C5E9002386
:10082000012007E0282C10D005D8012C09D0052C78
:100830000FD0002070BD302CFBD10BA3D3E90023D7
:10084000ECE70BA3D3E90023E8E70BA3D3E90023EC
:10085000E4E70BA3D3E90023E0E700BFAFF3008098
:10086000401DA12026812A0B78F6339F93CACD8D97
:100870009E6AC421818A46EE26417272DF25D7B76F
:10088000F017304A39059E5638B505460E4C002102
:10089000013500F0E5FBA4F82C55B4F82C0500F068
:1008A000C7FB78B1B4F82C0500F0D2FB014648B97B
:1008B000B4F82C0500F0D4FBB4F82C350133A4F8BF
:1008C0002C35EAE738BD00BFB044002010B50A4B14
:1008D0000A4A1A6003F5805393F860203AB9DC6D38
:1008E0002CB1204600F0EAFE204604F035F8BDE8C1
:1008F0001040034800F0E2BED83300203C4B000813
:10090000204400202DE9F04F8FB000AF05460C4683
:1009100002F0A6F8002849D1237E022B1BD1E38ADE
:10092000012B18D101F078FD0646FFF7E1FD0346E3
:100930004FF4C870DFF8C482B3FBF0F206F5167608
:1009400002FB103316FA83F3C8F80030E37E33B9A4
:10095000A34B00221A703C37BD46BDE8F08F07F16B
:100960002401204600F0D4FC0028F4D107F1140043
:10097000FFF7D6FD97F8264007F11401224607F14C
:10098000270004F033F80028E2D10F2C08D8944B4C
:100990001C70D8F80030A3F51673C8F80030DAE7F9
:1009A00097F82410284602F053F8D4E7E38A282B5E
:1009B0002BD010D8012B23D0052BCCD1BFF34F8FD8
:1009C0008849894BCA6802F4E0621343CB60BFF3E5
:1009D0004F8F00BFFDE7302BBDD1844EE17E327AD0
:1009E0009142B8D1607E3146002291F8DC508542B8
:1009F00000F0A5800132042A01F58A71F5D1AAE739
:100A000021462846FFF79CFDA5E721462846FFF72B
:100A100003FEA0E7B2F8EC507B6005F103094FEA52
:100A200099094FEA8902D11DC908A8EBC1039D4667
:100A3000EB460021584600F051FB04F1EE012A4636
:100A40003144584600F038FB7B6813B9012000F0B0
:100A5000E5FA96F8D20000F0EBFA044630B93072AD
:100A600000F006FB204600F0D9FAB1E0D6F8D42019
:100A70003AB996F8D200B6F82C25824201D8FFF791
:100A800003FFD6F8D4202A44944208D296F8D20024
:100A9000B6F82C250130824201D8FFF7F5FE7068C8
:100AA0005FFA89F2594600F021FB08B9C54679E0A2
:100AB000726896F8D2002A447260D6F8D42005EB0A
:100AC0000209C6F8D49000F0B3FA814509D396F82C
:100AD000D220D6F8D4000132001B86F8D220C6F806
:100AE000D400FF2D0FD80024347200F0C1FA204644
:100AF00000F094FA00F064FD3D4B188108B9FFF74F
:100B0000A3FCC54627E7BB6896F8D9000AFB036239
:100B1000FB68D2F8E41082F8E83001F58061C2F891
:100B2000E030C2F8E410FFF7D5FDFFF723FE96F89A
:100B3000D920013202F0030286F8D920B6E74FF43B
:100B40008A7A0AFB02F505F1EA013144204600F0F9
:100B5000B5FCF86000287FF4FEAE3544012285F82C
:100B6000E82001F059FCD5F8E020D6ED007ADFED61
:100B7000216A801A192838BF192040F6B8329042ED
:100B800028BF1046B8EE677A07EE900AF8EEE77ACB
:100B900067EEA67ADFED186AE7EE267AFCEEE77AD2
:100BA000C6ED007A96F8D930BB60BA6873680AFB64
:100BB00002F4321992F8E81059B1D2F8E4108B42DD
:100BC000E8463FF427AF002182F8E810C2F8E010B1
:100BD000C5467368064A9B0A01331381BBE600BF12
:100BE0009D33002000ED00E00400FA05B044002031
:100BF0008C230020CDCCCC3D6666663FA033002020
:100C0000014B1870704700BF9823002030B54FF09B
:100C100000542B4B22689A4285B007D003F0D6F8D7
:100C2000044620BB0024204605B030BD254B627D24
:100C300025481A70237D03724FF48073C0F8F83191
:100C40004FF40073C0F80C3300254FF44073C0F824
:100C500020341E49C0F8E450C922093000F02CFAB3
:100C60002046E022294600F039FA0124DBE7184A41
:100C7000184D136C43F000731364AA6D164B9A421F
:100C8000D0D12B6E013B7E2BCCD8144A07CA01ABC6
:100C900083E807001846032100F060FC6B6D834277
:100CA0004FF00003BED12A6D8A4201BFAB65054BF0
:100CB0002A6E1A7003BF0A4BEA6D1A601C46B2E72F
:100CC0009AAD44C598230020B044002016000020AF
:100CD00000380240006600405041A0B05866004015
:100CE0001023002037B51A4D00F06AFC02236B7107
:100CF000184B288119681848012201F029FA0023AD
:100D00000193164B164900931648174B4FF4805227
:100D100001F076FE154B197811B1124801F098FEDA
:100D200001F07AFB0446FFF7E3FB4FF4C873B0FB16
:100D3000F3F202FB130304F5167010FA83F00C4B68
:100D4000186003F039F808B10F232B8103B030BDD0
:100D50008C23002010230020D83300200108000835
:100D60009C230020A43300200509000898230020BC
:100D7000A03300202DE9F04F2DED028B0FF2382922
:100D8000D9E90089834C93B00BAE9FED7E8BFFF7C2
:100D9000F1FC814FDFF828A200230A93ADF834302C
:100DA0000B9373604FF0000B5B468DED008B0125BC
:100DB0000DF11D0207A938468DF81C508DF81DB0A5
:100DC00001F074F99DF81C30002B40F0A5802046FE
:100DD00001F046FE0646002845D1704F01F01CFB8D
:100DE0003B6898423FD301F017FB8246FFF780FB38
:100DF0004FF4C873B0FBF3F202FB13030AF516704D
:100E000010FA83F03860664F97F800B0CBF1100A03
:100E1000BBF1000F14BF33462B465FFA8AFA0EA8C7
:100E20008DF82830FFF77CFBBAF1060F28BF4FF092
:100E3000060A0EAB03EB0B0152460DF1290000F040
:100E40003BF90AAB0393182302930AF10102554BB5
:100E5000D2B2CDE90053049220464CA3D3E900233B
:100E600001F044FE3E7001F0D7FA4F4A4F4D13682F
:100E7000C31AB3F57A7F2ED3106001F0CFFA024681
:100E80000B46204601F0CAFE204601F0E9FD10B3F2
:100E90002B7A474E002B14BF03230223737101F0FA
:100EA000BBFA0EAF4FF47A730122B0FBF3F0394670
:100EB0003060304600F004FA182302933D4B019352
:100EC00080B240F25513CDE90370009342464B4681
:100ED000204601F00BFE2B7A93B101F09DFA00261B
:100EE00007464FF48A7A95F8D900304400F00300A1
:100EF0000AFB005393F8E82092B30136042EF2D196
:100F0000C82002F0DDFB2B7A002B7FF43DAF13B03D
:100F1000BDEC028BBDE8F08FDAF8143083F4805317
:100F2000CAF81430594610220EA800F0D7F80DF177
:100F30001E0308AA0AA9384600F020FE96E803001E
:100F40000FAB83E803009DF834308DF844300A9BE2
:100F50000E930EA9DDE90823204602F033F821E7BD
:100F6000D3F8E02042B12B68FA2B38BFFA23BA1A23
:100F70000533B2EB430FC0D3FFF7ACFB0028BCD165
:100F8000BEE700BF0000000000000000401DA120DF
:100F900026812A0BA4330020D8330020A033002060
:100FA0009D3300209C330020E0490020B044002005
:100FB0008C230020E4490020F1C6A7C1D068080FA7
:100FC0000004024008B5054800F074FEBDE8084082
:100FD000034A0449002003F0B9BC00BFD833002005
:100FE000204A0020CD08000870B502F03DFD094EF2
:100FF000094D3080002428683388834208D902F0E4
:101000002DFD2B6804440133B4F5803F2B60F2D3EF
:1010100070BD00BF144A0020E849002002F0D4BD92
:1010200000F10060920000F5803002F063BD000026
:10103000054B1A68054B1B889B1A834202D9104442
:1010400002F00CBD00207047E8490020144A00203F
:10105000024B1B68184402F009BD00BFE84900209C
:10106000024B1B68184402F019BD00BFE84900207C
:10107000064991F8243033B10023086A81F82430FE
:101080000822FFF7CDBF0120704700BFEC490020C8
:10109000022802BF024B4FF480529A61704700BF92
:1010A00000040240022802BF024B4FF080529A61B6
:1010B000704700BF0004024010B50023934203D0E4
:1010C000CC5CC4540133F9E710BD0000034602466E
:1010D000D01A12F9011B0029FAD1704702440346C5
:1010E000934202D003F8011BFAE770472DE9F84359
:1010F0001F4D144695F824200746884652BBDFF85A
:1011000070909CB395F824302BB92022FF214846DB
:101110002F62FFF7E3FF95F82400C0F10802A24216
:1011200028BF2246D6B24146920005EB8000FFF769
:10113000C3FF95F82430A41B1E44F6B2082E1744B2
:101140009044E4B285F82460DBD1FFF791FF0028DA
:10115000D7D108E02B6A03EB82038342CFD0FFF79D
:1011600087FF0028CBD10020BDE8F8830120FBE7F2
:10117000EC4900202DE9F0470D4604460021904639
:10118000284640F27912FFF7A9FF234620220021CA
:10119000284601F0B9FE231D02222021284601F035
:1011A000B3FE631D03222221284601F0ADFEA31DDC
:1011B00003222521284601F0A7FE04F1080310228E
:1011C0002821284601F0A0FE04F11003082238214E
:1011D000284601F099FE04F1110308224021284617
:1011E00001F092FE04F1120308224821284601F082
:1011F0008BFE04F1140320225021284601F084FEC6
:1012000004F1180340227021284601F07DFE04F10C
:1012100020030822B021284601F076FE04F12103C4
:101220000822B821284601F06FFE04F12207C026EB
:101230003B46314608222846083601F065FEB6F5E1
:10124000A07F07F10107F3D104F1320308223146F0
:10125000284601F059FE002704F1330A94F8323091
:101260004FEAC7099F4209F5A47615D3B8F1000FDC
:1012700008D1314604F599730722284601F044FE4F
:1012800009F24F16274694F832213B1B93420CD3A8
:10129000F01DC008BDE8F0870AEB070308223146BD
:1012A000284601F031FE0137D8E707F23313314603
:1012B0000822284601F028FE08360137E3E700003F
:1012C00013B504460846002101602346C0F8031008
:1012D0002022019001F018FE0198231D02222021F6
:1012E00001F012FE0198631D0322222101F00CFE81
:1012F0000198A31D0322252101F006FE019804F1A7
:1013000008031022282101F0FFFD072002B010BDC4
:10131000F7B50023047F00910E46072219460546C3
:1013200001F0B6FC731C009301220023072128461C
:1013300001F0AEFCC4B9B31C00930522234608217A
:10134000284601F0A5FC0D243746B278BB1B93421A
:1013500011D32B7FA88A0734E408BBB9844294BF19
:101360000020012003B0F0BDAB8ADB00083BDB08A6
:10137000B3700824E8E7FB1C0093214600230822F1
:10138000284601F085FC08340137DEE7201A18BF33
:101390000120E7E7F7B50023047F00910E460822FD
:1013A0001946054601F074FC731CC4B90822009369
:1013B00011462346284601F06BFC10240123727865
:1013C0005F1C013B934211D32B7FA88A0734E408AA
:1013D000BBB9844294BF0020012003B0F0BDAB8AAA
:1013E000DB00083BDB0873700824E7E7F319009380
:1013F000214600230822284601F04AFC08343B46D7
:10140000DDE7201A18BF0120E7E70000F8B50E4617
:1014100005461446002181223046FFF75FFE2B4629
:1014200008220021304601F06FFD7CB96B1C0722B9
:101430000821304601F068FD0F2401236A785F1C03
:10144000013B934204D3E01DC008F8BD0824F4E733
:10145000EB1921460822304601F056FD08343B4680
:10146000ECE70000F8B50E46054614460021CE22F2
:101470003046FFF733FE2B4628220021304601F08C
:1014800043FD7CB905F1080308222821304601F00C
:101490003BFD30242F462A7A7B1B934204D3E01D68
:1014A000C008F8BD2824F5E707F109032146082202
:1014B000304601F029FD08340137ECE7F7B5047F29
:1014C00000910E46012310220021054601F0E0FBA9
:1014D000C4B9B31C0093092223461021284601F009
:1014E000D7FB192437467288BB1B9A4211D82B7F31
:1014F000A88A0734E408BBB9844294BF00200120C5
:1015000003B0F0BDAB8ADB00103BDB087380102416
:10151000E8E73B1D0093214600230822284601F0FE
:10152000B7FB08340137DEE7201A18BF0120E7E7D0
:1015300030B5094D0A4491420DD011F8013B584095
:10154000082340F30004013B2C4013F0FF0384EA1E
:101550005000F6D1EFE730BD2083B8EDF7B54FF07E
:10156000FF33DFF854C0DFF854E000EB81011A4686
:1015700088421CD050F8044B019401AF042417F8A2
:10158000015B82EA05620825DB18164605F1FF3586
:101590005241002EBCBF83EA0C0382EA0E0215F012
:1015A000FF05F1D1013C14F0FF04E8D1E0E7D84396
:1015B000D14303B0F0BD00BF9336EAA9EBE1F0429E
:1015C000F7B5384A106851686B4603C36A46364916
:1015D0003648082303F01AFA0446002833D10A25B6
:1015E000334A106851686B4603C36A4631492F4835
:1015F000082303F00BFA0446002849D00369B3F529
:10160000E02F45D8B0F8661040F2E93291423FD160
:10161000294A024402F15C018B4239D35C3B2349E5
:1016200000209E1AFFF784FF3246074604F164014A
:101630000020FFF77DFFA3689F4229D1E36898420D
:1016400008BF002524E00369B3F5E02F27D8418BBC
:1016500040F2E932914220D1174A024402F11001CE
:101660008B4218D3103B114900209D1AFFF760FFF1
:101670002A46064604F118010020FFF759FFA36827
:101680009E4202D1E368984201D00D25A8E70025CB
:10169000284603B0F0BD1025A2E70C25A0E70B25D6
:1016A0009EE700BF004B0008DCFF060000000108B9
:1016B000094B000890FF06000800FFF710B5037CF7
:1016C000044613B9006803F089F9204610BD0000F4
:1016D0000023BFF35B8FC360BFF35B8FBFF35B8FF0
:1016E0008360BFF35B8F7047BFF35B8F0068BFF30E
:1016F0005B8F704770B505460C30FFF7F5FF05F1BD
:10170000080604463046FFF7EFFFA04206D93046F0
:101710006D68FFF7E9FF2544281A70BD3046FFF7D2
:10172000E3FF201AF9E7000070B50546406898B15C
:1017300005F10800FFF7D8FF05F10C060446304616
:10174000FFF7D2FF8442304694BF6D680025FFF753
:10175000CBFF013C2C44201A70BD000038B50C466C
:101760000546FFF7C7FFA04210D305F10800FFF7B9
:10177000BBFF04446868B4FBF0F100FB1144BFF305
:101780005B8F0120AC60BFF35B8F38BD0020FCE7AE
:101790002DE9F041144607460D46FFF7C5FF844288
:1017A00028BF0446D4B1B84658F80C6B4046FFF742
:1017B0009BFF3044286040467E68FFF795FF331A50
:1017C0009C4203D86C600120BDE8F0816B60A41BD3
:1017D0003B68AB602044E8600220F5E72046F3E771
:1017E00038B50C460546FFF79FFFA04210D305F120
:1017F0000C00FFF779FF04446868B4FBF0F100FBCC
:101800001144BFF35B8F0120EC60BFF35B8F38BDE9
:101810000020FCE72DE9FF41884669460746FFF7AF
:10182000B7FF6C4606B204EBC6060025B44209D0E9
:101830006268206808EB0501FFF73EFC6368083426
:101840001D44F3E729463846FFF7CAFF284604B08F
:10185000BDE8F081F8B505460C300F46FFF744FFB0
:1018600005F1080604463046FFF73EFFA042304629
:1018700088BF6C68FFF738FF201A386020B1304607
:101880002C68FFF731FF2044F8BD000073B5144603
:1018900006460D46FFF72EFF844228BF04460190FE
:1018A000DCB101A93046FFF7D5FF019B33B932689F
:1018B000C5E90233C5E9002401200CE09C4238BF91
:1018C00001942860019868608442F5D93368AB6060
:1018D000241AEC60022002B070BD2046FBE7000035
:1018E0002DE9FF410F466946FFF7D0FF6C4600B275
:1018F00004EBC0050026AC4209D0D4F8048054F8AB
:10190000081BB8194246FFF7D7FB4644F3E73046B9
:1019100004B0BDE8F081000038B50546FFF7E0FFF0
:10192000044601462846FFF719FF204638BD00004F
:1019300010B4026854681A4623465DF8044B1847F1
:10194000002070470020704770470000002070475B
:101950000E20704700F5805090F8C800C0F340009A
:101960007047000000F5805090F9D00070470000EB
:1019700000F58050C0F8CC1001207047F7B50C6816
:10198000BDF8207014F0005470D10D7B082D6DD877
:10199000302585F311884569AE6876010CD4AC68B2
:1019A000240108D4AC6814F080545DD184F311880C
:1019B000204603B0F0BD01240E6804F1180C002E7F
:1019C000B8BFF6004FEA0C1CB4BF46F0040676051B
:1019D00045F80C600E680FFA84FC16F0804F18BFB3
:1019E00005EB0C1E05EB0C1C1EBFDEF8806146F0FB
:1019F0000206CEF880610E7BCCF8846105EB0415FD
:101A00008E68C5F88C614E68C5F88861DCF8805135
:101A100045F00105CCF8805100EB441641F2680511
:101A20002E4405EB44150544C6E9002308350E464F
:101A300001F10C0C56F804EB45F804EB6645F9D1BE
:101A4000843436882E8000EB441407F00305267991
:101A500026F00B0635432571002484F31188009786
:101A600000F0FCFC0120A4E70224A5E74FF0FF30C2
:101A70009FE7000013B500F580540191E06DFFF77A
:101A800053FE1F280AD90199E06D2022FFF7C2FEFC
:101A9000A0F120035842584102B010BD0020FBE7DE
:101AA00008B5302383F3118800F58050C06DFFF72F
:101AB0000FFE002383F3118808BD0000002202609E
:101AC000828142608260704710B500220023C0E925
:101AD00000230023044603810C30FFF7EFFF20466C
:101AE00010BD0000F0B5054600F580500C4690F89A
:101AF000C83013F0040FC3F3800108BF114661F32F
:101B0000820304F1840680F8C83005EB461389B0DF
:101B10001B79D8072ED57AB319072DD46846FFF75D
:101B2000D3FF05EB441303F5835303F1180703AA0E
:101B3000103318685968144603C40833BB42224660
:101B4000F7D1186820609B88A380DDE90E23CDE9DA
:101B500000230123ADF808302B686946DB6B28466B
:101B6000984705EB46152B791A075CBF43F008032D
:101B70002B7101E0002AF4D109B0F0BD2DE9F04746
:101B80009A4688B0074688469146302383F31188E9
:101B900007F580546846FFF797FFE06DFFF7AAFD51
:101BA0001F282AD9E06D20226946FFF7B5FE2028BC
:101BB00023D103AD444605AB2E4603CE9E422060A2
:101BC0006160354604F10804F6D130682060B388BE
:101BD000A380DDE90023C9E90023BDF80830AAF895
:101BE0000030002383F3118853464A464146384665
:101BF00008B0BDE8F04700F01FBC002080F311885A
:101C000008B0BDE8F08700002DE9F84F0023C0E9D7
:101C10000133254B044640F8183B0F46FFF74EFFB3
:101C200004F12800FFF750FF04F1480804F582553D
:101C30004646083530462036FFF746FFAE42F9D11A
:101C400004F580554FF480534FF00009C5E913396E
:101C5000C5F848800123EE6504F5875804F58456DD
:101C6000C5F8549085F8583085F86030083608F18A
:101C700008084FF0000A4FF0000B46E908ABA6F148
:101C80001800FFF71BFF203646F8289C4645F4D184
:101C900085F8D07017B1054800F0B8FB044B6361BC
:101CA0002046BDE8F88F00BF3C4B0008144B0008ED
:101CB0000064004010B5044B197804464A1C1A70A1
:101CC000FFF7A2FF204610BD1C4A00202DE9F04777
:101CD000002950D0294B2A4FB7FBF1F599428CBF10
:101CE0000A231123581EB5FBF3FC03FB1C53C4B29B
:101CF0002BB102280346F5D80020BDE8F0870CF18F
:101D0000FF36B6F5806FF7D2C4EBC40E0EF10303B5
:101D10004FEAE309C3F3C703A4EB030809F1010A7F
:101D20004FF47A755FFA88F009FB05555AFA88F87E
:101D3000B5FBF8F5B5F5617FC1BF0EF1FF33C3F315
:101D4000C703E01AC0B25C1C50FA84F40CFB04F424
:101D5000B7FBF4F4A142CFD1013BDBB20F2BCBD8C0
:101D60000138C0B20728C7D80021107116809170C1
:101D7000D3700120C1E70846BFE700BF3F420F0014
:101D800040787D0170B505460E464FF47A746B6954
:101D90005B6803F00103B34207D04FF47A7001F09F
:101DA0008FFC013CF3D1204670BD0120FCE7000010
:101DB00030B54269936913F0700F16D000230B4CB5
:101DC000936103F1840200EB421211794D0709D5AA
:101DD000890707D5416954F823508D60117941F086
:101DE000040111710133032BEBD130BD284B0008E6
:101DF00073B51D46436916469A68D207044609D54D
:101E00009A6801219960C2F34002CDE90065002182
:101E1000FFF768FE63699A68D1050BD59A684FF49D
:101E200080719960C2F34022CDE90065012120460E
:101E3000FFF758FE63699A68D2030BD59A684FF48E
:101E400080319960C2F34042CDE90065022120460D
:101E5000FFF748FE04F58053D3F8CC0010B10368B7
:101E60001B699847204602B0BDE87040FFF7A0BF4D
:101E7000F8B504464669002972D106F10C073868A6
:101E8000800770D006EB01153868D5F8B00110F066
:101E9000040FD5F8B0011ABFC00840F00040400D53
:101EA000A061D5F8B0C11CF0020F1CBF40F080400B
:101EB000A061D5F8B40106EB011100F00F0084F821
:101EC0002400D1F8B8012077D1F8B801000A607772
:101ED000D1F8B801000CA077D1F8B801000EE07776
:101EE000D1F8BC0184F82000D1F8BC01000A84F8C4
:101EF0002100D1F8BC01000C84F82200D1F8BC11FB
:101F0000090E84F823103821396004F1340004F1FB
:101F1000180104F1240551F8046B40F8046BA94240
:101F2000F9D109880180C4E90A23214600232386C8
:101F300051F8283B2046DB6B984704F5805393F813
:101F4000C820D3F8CC0042F0040283F8C82010B1B6
:101F500003681B6998472046BDE8F840FFF728BF93
:101F600006F110078BE7F8BD10B5044600F056FAED
:101F700002460B4652EA030102D0013A63F1000324
:101F80000449086820B12146BDE81040FFF770BF42
:101F900010BD00BF184A0020F0B5302181F3118830
:101FA000DFF848C000F583510831002404F18405AE
:101FB00000EB45152E7977070ED4F6060CD5D1E93E
:101FC000007697429E4107D246695CF82470B7605C
:101FD0002E7946F004062E710134032C01F1200104
:101FE000E4D1002383F31188F0BD00BF284B000823
:101FF00008B5302383F31188FFF7DAFE002383F35B
:10200000118808BDF8B543690546986800F0E050AE
:10201000B0F1E05F0F4621D0F8B1302383F311888F
:1020200005F583541034002606F1840305EB4313B1
:102030001B791A0706D50136032E04F12004F3D1CB
:10204000012007E05B07F6D42146384600F040FA4D
:102050000028F0D1002383F31188F8BD0120FCE7AC
:1020600008B5302383F3118800F58050C06DFFF769
:1020700041FB002383F3118843090CBF012000209A
:1020800008BD0000F8B51D46002313700F46064634
:102090001446FFF7E5FF80F00100387025B12946AE
:1020A0003046FFF7AFFF2070F8BD00002DE9B841C2
:1020B0000C4615461F46804600F0B0F90B462178C5
:1020C000024609B9287850B14046FFF765FFFFF78F
:1020D0008FFF3B462A462146FFF7D4FF0120BDE88B
:1020E000B881000070B5302686F31188174B1A6C42
:1020F00042F000721A641A6A42F000721A621A6A96
:1021000022F000721A62002383F3118800F58054D4
:1021100094F8C83013F0010516D1A9B186F31188DF
:102120000321132001F0C8F90321142001F0C4F9A0
:102130000321152001F0C0F994F8C83043F00103E1
:1021400084F8C83085F3118870BD00BF00380240A4
:102150002DE9F04700F5805588B095F8D030012B77
:1021600004468846164600F28180814F57F82320A6
:102170000AB947F82300D7F800A0C4F80C802674E9
:10218000BAF1000F64D095F8D030012B70D0012146
:102190002046FFF7A7FF302383F311886269136895
:1021A00023F0020313606269136843F001031360B4
:1021B000636900275F6187F3118801212046FFF7DB
:1021C000E1FD002800F09580E86DFFF781FA04F545
:1021D0008359BA4609F10809202200216846FEF712
:1021E0007DFF02A8FFF76AFCCDF818A06A4609EB4C
:1021F00007030DF1180E9446BCE80300F44518607F
:102200005960624603F10803F5D1DCF8000018605C
:1022100020379CF804201A71602FDDD195F8C83062
:102220006FF38203002785F8C8306A46414620468E
:10223000ADF80070ADF802708DF80470FFF746FD40
:10224000636948BB4FF400421A6008B0BDE8F087EC
:1022500041F2D80002F082FB814610B15146FFF7EF
:10226000D3FCC7F80090B9F1000F8CD10020ECE747
:10227000386803681B6B98470146002887D1386887
:10228000FFF730FF3868036832465B68414698477D
:1022900000287FF47CAFE9E761221A609DF80230E4
:1022A0009DF803201B06120402F4702203F0407311
:1022B0001343BDF80020C2F3090213439DF8042024
:1022C0001205022E02F4E0020CBF4FF00041002183
:1022D000134362690B43D361636913225A616269D4
:1022E000136823F00103136039462046FFF74AFDC7
:1022F00008B96369A6E795F8D03093BB6169D1F856
:10230000002242F00102C1F800226169D1F80022E6
:1023100022F47C5222F00E02C1F800226169D1F849
:10232000002242F46062C1F800226269C2F81432ED
:102330006269C2F80432626941F6FF71C2F80C1298
:102340006269C2F840326269C2F8443263690122AC
:10235000C3F81C226269D2F8003223F00103C2F8EC
:10236000003295F8C83043F0020385F8C8306CE7B6
:10237000184A002008B500F051F850EA010302465F
:1023800002D0421E61F10001044B186810B10B46E7
:10239000FFF72EFDBDE8084001F064B8184A0020A0
:1023A00008B50020FFF7E0FDBDE8084001F05AB88D
:1023B00008B50120FFF7D8FDBDE8084001F052B88C
:1023C00000B59BB0EFF3098168226846FEF774FE02
:1023D000EFF30583014B9B6BFEE700BF00ED00E0D0
:1023E00008B5FFF7EDFF000000B59BB0EFF30981E2
:1023F00068226846FEF760FEEFF30583014B5B6BD6
:10240000FEE700BF00ED00E0FEE700000FB408B5F6
:10241000029801F005F9FEE701F01ABC01F0FCBBDF
:1024200013B56C4684E80600031D94E8030083E8B6
:102430000500012002B010BD73B58568019155B14A
:102440001B885B0707D4D0E900369B6B9847019A3D
:10245000C1B23046A847012002B070BDF0B5866811
:1024600089B005460C465EB1BDF838305B070AD42A
:10247000D0E900379B6B98472246C1B23846B04737
:10248000012009B0F0BD00220023CDE90023002384
:10249000ADF808300A4603AB01F108061068516830
:1024A0001C4603C40832B2422346F7D110682060AC
:1024B0009288A280FFF7B2FF0423ADF808302B68A2
:1024C000CDE90001DB6B694628469847D8E7000054
:1024D00030B503680968DD0FB5EBD17F23F06044A8
:1024E00021F060424FEAD1700BD0002BB8BFA40C92
:1024F0000029B8BF920C944202D034BF01200020C2
:1025000030BD944205D1C1F38070C3F38073834220
:10251000F6D194422CBF00200120F1E72DE9F041D3
:10252000456A15B94162BDE8F0814B6823F0604708
:10253000C3F38A464FEAD37EC3F3807816EA2306B4
:1025400038BF3E46AC462B465A68BEEBD27F22F0DF
:1025500060440AD0002A18DAA40CB44217D19D4274
:102560000FD10D60DEE71346EEE7A74207D102F078
:102570008044C2F3807242450BD054B1EFE708D2D9
:10258000EDE7CCF800100B60CDE7B44201D0B442C7
:10259000E5D81A689C46002AE5D11960C3E7000017
:1025A0002DE9F047089D01F007044FEAD5082244C1
:1025B00005F0070500EBD1004FF47F49944201D1AB
:1025C000BDE8F08704F0070705F0070A57453E46C7
:1025D00038BF5646C6F10806111B8E4228BF0E466C
:1025E000E10808EBD50E415C13F80EC0B94029FA9A
:1025F00006F721FA0AF1FFB28CEA010147FA0AF75D
:1026000039408CEA010C03F80EC034443544D5E758
:1026100080EA0120082341F2210201B24000002992
:1026200080B203F1FF33B8BF504013F0FF03F4D181
:102630007047000038B50C468D18A54200D138BD52
:1026400014F8011BFFF7E4FFF7E7000042684AB106
:10265000136843604389818901339BB29942438166
:1026600038BF83811046704770B588B02022044679
:102670000D4668460021FEF731FD20460495FFF720
:10268000E5FF024658B16B46054608AE1C4603CC32
:10269000B44228606960234605F10805F6D110466A
:1026A00008B070BD082817D909280CD00A280CD00A
:1026B0000B280CD00C280CD00D280CD00E2814BFE1
:1026C0004020302070470C207047102070471420A5
:1026D000704718207047202070470000082817D93D
:1026E0000C280CD910280CD914280CD918280CD96E
:1026F00020280CD930288CBF0F200E2070470920CD
:1027000070470A2070470B2070470C2070470D203F
:10271000704700002DE9F843078C072F04461ED9A7
:10272000D0E9029800254FF6FF73C5F12006A5F108
:10273000200029FA05F108FA06F628FA00F03143DC
:102740000143C9B21846FFF763FF0835402D034621
:10275000EBD1E1693A46BDE8F843FFF76BBF4FF6AE
:10276000FF70BDE8F883000010B54B6823B9CA8A32
:1027700063F30902CA8210BD04691A681C60036110
:10278000C38A013BC3824A60EFE700002DE9F84F9E
:102790001D46CB8A0F46C3F309010529814692469F
:1027A0000B4630D00020AAB207F11A049EB2042EC4
:1027B0001FFA80F80FD8904503F1010306D3FB8A76
:1027C0000A4462F30903FB8201201AE01AF8006050
:1027D000E6540130EAE79045F1D2A1F1050B1C2344
:1027E0007C68BBFBF3F203FB12BB1FFA8BF6002CD9
:1027F00045D14846FFF72AFF044638B978606FF0A4
:102800000200BDE8F88F4FF00008E6E700260660FA
:102810007860ADB24FF0000B454510D90AEB0803C4
:10282000221D13F8011B9155B1B208F101081B29B3
:102830001FFA88F82BD0454506F10106F1D8FB8A2E
:10284000C3F30902154465F30903BCE7013292B2F0
:102850001C462368002BF9D16B1F0B441C21B3FBD2
:10286000F1F301339BB29A42D3D2BBF1000FD0D126
:102870004846FFF7EBFE20B9C4F800B0BFE70122DD
:10288000E7E7C0F800B05E4620600446C1E7454572
:10289000D5D94846FFF7DAFE08B92060AFE7C0F89F
:1028A00000B0002620600446B6E700002DE9F04F96
:1028B0002DED028B1C4683B05B690192074688466A
:1028C000002B00F09A80238C2BB1E269002A00F0E3
:1028D0009480072B35D807F10C00FFF7B7FE0546AB
:1028E00038B96FF00205284603B0BDEC028BBDE895
:1028F000F08F14220021FEF7F1FB228CE16905F133
:102900000800FEF7D9FB208C013080B2FFF7E6FE0D
:10291000FFF7C8FE013880B2208401302874636953
:10292000228C1B782A4403F01F0363F03F0348F016
:1029300000411372384669602946FFF7EFFD012513
:10294000D1E700F10C034FF0000908EE103A4FF008
:10295000800A4E464D4618EE100AFFF777FE834672
:102960000028BED014220021FEF7B8FB002E3AD179
:10297000019BABF8083002220BF1080E1FFA82FC13
:102980000CF10100BCF1060F218C80B201D88E42FF
:102990002BD3FFF7A3FEFFF785FE6269127801389B
:1029A00002F01F028E4208BF4FF0400A42EA49126D
:1029B0001BFA80F14AEA020A013048F0004281F82D
:1029C00008A08BF81000CBF8042059463846FFF7D2
:1029D000A5FD238C0135B3422DB289F001094FF0DA
:1029E000000AB8D17FE70022C6E7E169895D0EF8E9
:1029F00002100136B6B20132C0E76FF0010572E78E
:102A0000F8B515460E463022002104461F46FEF753
:102A100065FB069B6360B5F5001F079BA76034BF8D
:102A20006A094FF6FF72A36297B2E66104F11000E3
:102A300000239A4206D800230360A782E3822383FF
:102A4000E360F8BD0660013330462036F1E7000050
:102A500003781BB94BB2002BC8BF01707047000050
:102A600000787047F8B50C46C969074611B9238C40
:102A7000002B37D1257E1F2D34D8387828BB228CE7
:102A8000072A2CD8268A36F003032BD14FF6FF7085
:102A9000FFF7D0FD20F001003102400441EA05615A
:102AA000400C41EA40254FF6FF722346294638463E
:102AB000FFF7FCFE002807DD626913780133DBB203
:102AC0001F2B88BF00231370F8BD218A2D0645EA0D
:102AD000012505432046FFF71DFE0246E5E76FF09E
:102AE0000300F1E76FF00100EEE7000070B58AB077
:102AF000044616460021282268461D46FEF7EEFAD7
:102B0000BDF83830ADF810300F9B05939DF840307C
:102B10008DF81830119B07936946BDF84830ADF821
:102B200020302046CDE90265FFF79CFF0AB070BD5A
:102B30002DE9F041D36905460C4616460BB9138CB6
:102B40005BBB377E1F2F28D895F80080B8F1000FA7
:102B500026D03046FFF7DEFD3378210241EAC3314B
:102B600041EA0801338A41EA076141EA034102462A
:102B7000334641F080012846FFF798FE00280ADD21
:102B80003378012B07D1726913780133DBB21F2B25
:102B900088BF00231370BDE8F0816FF00100FAE7F1
:102BA0006FF00300F7E70000F0B58BB004460D4668
:102BB00017460021282268461E46FEF78FFA9DF828
:102BC0004C305A1E534253418DF800309DF840302E
:102BD000ADF81030119B05939DF848308DF81830F2
:102BE000149B07936A46BDF85430ADF8203029464F
:102BF0002046CDE90276FFF79BFF0BB0F0BD000049
:102C0000406A00B104307047436A1A684262026940
:102C10001A600361C38A013BC38270472DE9F0410A
:102C2000D0F82080194E14461D464146002709B9A8
:102C3000BDE8F081D1E90223A21A65EB03039642B5
:102C400077EB03031ED2036A8B420DD1FFF78CFD95
:102C5000036A1B68036203690B60C38A0161016A2E
:102C6000013BC3828846E2E7FFF77EFD0B68C8F8A8
:102C7000003003690B60C38A0161013BC382D8F84D
:102C80000010D4E788460968D1E700BF80841E00A1
:102C90002DE9F04F8BB00D46DDF8509014469B4661
:102CA0008046002800F01981B9F1000F00F015816D
:102CB000531E3F2B00F21181012A03D1BBF1000FFB
:102CC00040F00B810023CDE90833B8F81430B5EBA0
:102CD000C30F4FEAC30703D300200BB0BDE8F08F4A
:102CE0002B199F42D8F80C303ABF7F1BFFB2274602
:102CF0001BB9D8F81030002B7AD0272D4ED8C5F14B
:102D00002806B7424FF000032CBFF6B23E460093B0
:102D10002946D8F8080008AB3246FFF741FCA7EB7C
:102D2000060A35445FFA8AFAB8F8143003F1005302
:102D3000053BDB000493D8F80C3003932821039B58
:102D400013B1BAF1000F2CD1D8F8100040B1BAF18C
:102D5000000F05D0009608AB5246691AFFF720FC19
:102D600038B2002FB8D066070AD00AAB03EBD40103
:102D7000624211F8083C02F00702134101F8083CD6
:102D8000082C3CD9102C40F2B580202C40F2B780A2
:102D9000BBF1000F00F09C80082334E0BA46002607
:102DA000C2E7049BE02B28BFE02306930B44AB4211
:102DB000059314D95A1B03980096924534BF524686
:102DC000D2B2691A08AB04300792FFF7E9FB079A01
:102DD0001644AAEB020A1544F6B25FFA8AFA049B7B
:102DE000069A05999B1A0493039B1B680393A6E715
:102DF0000093D8F8080008AB3A462946AEE7BBF185
:102E0000000F13D00123B4EBC30F6CD0082C12D8E1
:102E10009DF82030621E23FA02F2D50706D54FF046
:102E2000FF3202FA04F423438DF820309DF820305D
:102E300089F8003051E7102C12D8BDF82030621EFE
:102E400023FA02F2D10706D54FF0FF3202FA04F45A
:102E50002343ADF82030BDF82030A9F800303CE71E
:102E6000202C0FD80899631E21FA03F3DA0705D541
:102E70004FF0FF3202FA04F40C430894089BC9F89F
:102E800000302AE7402C2BD0DDE90865611EC4F133
:102E90002102A4F1210326FA01F105FA02F225FA32
:102EA00003F311431943CB0712D50122A4F12003E8
:102EB000C4F1200102FA03F322FA01F1A2405242C6
:102EC00043EA010363EB430332432B43CDE9082379
:102ED000DDE90823C9E90023FFE66FF00100FCE605
:102EE0006FF00800F9E6082CA0D9102CB3D9202CDB
:102EF000EED8C3E7BBF1000FADD0022383E7BBF1EF
:102F0000000FBBD004237EE730B5012A144638BF3A
:102F10000124402C85B028BF40240025012ACDE99A
:102F2000025518D81B788DF8083063070AD004AB17
:102F300003EBD405624215F8083C02F00702934007
:102F400005F8083C009103462246002102A8FFF73D
:102F500027FB05B030BD082AE4D9102A03D81B8806
:102F6000ADF80830E1E7202A8DBFD3E900231B68C4
:102F70000293CDE90223D8E710B5CB681BB98B606B
:102F80000B618B8210BD04691A681C600361C38ADF
:102F9000013BC382CA60F0E703064CBFC0F3C030F8
:102FA0000220704708B50246FFF7F6FF022806D157
:102FB0005306C2F30F2001D100F0030008BDC2F395
:102FC0000740FBE72DE9F04F93B0CDE903230A68F2
:102FD00004461046FFF7E0FF022814BFC2F306269E
:102FE0000026002A0D46824680F2F28112F0C04986
:102FF00040F0EE81097B002900F0EA81022803D02D
:103000002378B34240F0E781C2F30463069310468D
:1030100002F07F030593FFF7C5FF059B29444FEAA4
:10302000834848EA0A4848EA4668CE7800230022E6
:10303000CDE90823F309834648EA0008029367D0E4
:10304000059B009302466768534608A92046B84787
:10305000002800F0C381276A4FB9414604F10C00F3
:10306000FFF702FB074690B96FF0020054E03B699E
:1030700098450DD03F68002FF9D1414604F10C006E
:10308000FFF7F2FA07460028EED0236A3B6027627A
:1030900097F817C006F01F08CCF3840CACEB0800BF
:1030A0001FFA80FE0028B8BF0EF12000A8EB0C0329
:1030B0001FFA83FED7E90221B8BF00B2002B0793A5
:1030C000BEBF0EF120031BB2079352EA010338D0B2
:1030D000039BDFF824E39A1A049B4FF0000C63EB88
:1030E000010196457CEB01032BD36B7B97F81AE02B
:1030F000734519D1029B002B78D0012821DC786818
:10310000F8B9DFF8F0C2944570EB010316D337E04D
:10311000276A27B96FF00C0013B0BDE8F08F3B6948
:103120009845B5D03F68F4E7B24890427CEB010384
:1031300001D30020F0E7029B002BFAD0079B0F2B56
:1031400017DCFA7DB30002F0030203F07C031343A3
:10315000FB7539462046FFF707FB6B7BBB76029B6E
:103160003BB9FB7DC3F38402013262F38603FB7536
:10317000D0E76A7BBB7E9A42DBD1029B002B35D025
:10318000B309022B32D0039BBB60049BFB6014226B
:1031900000210DA8FDF7A2FF039B0A93049B0B934C
:1031A0002B1D0C932B7BADF83EB0013BDBB2ADF891
:1031B0003C30069B8DF84230059B8DF8433094F8E7
:1031C0002C308DF840A083F001038DF844308DF849
:1031D0004180A3680AA920469847FB7DC3F3840376
:1031E000013303F01F039B02FB82A2E7FB7DC6F3C2
:1031F0004012B2EBD31F40F0F480C3F38403434585
:1032000040F0F280029A2B7BB609002A4DD0F207DB
:103210005DD4032B40F2EB80039BBB60049BFB60FF
:103220002B7BAE1D033BDBB23246394604F10C006A
:10323000FFF7ACFA00280CDA39462046FFF794FA7B
:10324000FB7DC3F38403013303F01F039B02FB8266
:103250000AE7DDE90884AB883B834FF6FF73C9F1C9
:103260002000A9F1200228FA09F104FA00F0014334
:1032700024FA02F211431846C9B2FFF7C9F909F15D
:103280000809B9F1400F0346E9D1B8822A7B033A15
:10329000D2B23146FFF7CEF9FB7DB882DA43C2F3F2
:1032A000C01262F3C713FB7543E786B92E1D013BBD
:1032B000DBB23246394604F10C00FFF767FA00280A
:1032C000BADB2A7BB88A013AD2B23146E2E7F98A00
:1032D000C1F30901013B0429DAB25BD8281D0023A0
:1032E00007F11B069A4208D910F801CB06F801C075
:1032F000013101330529DBB2F4D103990A91049914
:103300000B91934207F11B010C9138BF043379688C
:103310000D9134BF55FA83F300230E93FB8AADF869
:103320003EB0C3F309031A44069B8DF84230059B57
:103330008DF8433094F82C30ADF83C2083F0010335
:103340008DF8443000238DF840A08DF841807B60DB
:103350002A7BB88A013A291DFFF76CF93B8BB882AA
:10336000834203D1A3680AA92046984720460AA9A8
:10337000FFF702FEFB7DBA8AC3F38403013303F037
:103380001F039B02FB823B8B9A420CBF00206FF015
:103390001000C1E67B68002BAFD0052001E01C3097
:1033A00033461E68002EFAD1091A081D2E1D184436
:1033B00001EB090CBCF11B0F5FFA89F39DD89A420F
:1033C0009BD916F8013B00F8013B09F10109EFE731
:1033D0006FF00900A0E66FF00A009DE66FF00B00A9
:1033E0009AE66FF00D0097E66FF00E0094E66FF02E
:1033F0000F0091E640420F0080841E00EFF3098326
:1034000005494A6B22F001024A63683383F3098855
:10341000002383F31188704700EF00E0302080F331
:10342000118862B60C4B0D4AD96821F4E061090499
:10343000090C0A43DA60D3F8FC20094942F0807293
:10344000C3F8FC200A6842F001020A602022DA7701
:1034500083F82200704700BF00ED00E00003FA058A
:10346000001000E010B5302383F311880E4B5B6829
:1034700013F4006314D0F1EE103AEFF30984683CC2
:103480004FF08073E361094BDB6B236684F309889B
:1034900000F090F810B1064BA36110BD054BFBE79F
:1034A00083F31188F9E700BF00ED00E000EF00E0D2
:1034B0003F0300084203000800F1604303F5614345
:1034C0000901C9B283F80013012200F01F039A40DA
:1034D00043099B0003F1604303F56143C3F8802176
:1034E0001A60704700230375826803691B68996836
:1034F0009142FBD25A680360426010605860704786
:1035000000230375826803691B6899689142FBD8A0
:103510005A680360426010605860704708B50846FA
:10352000302383F311880B7D032B05D0042B0DD0A2
:103530002BB983F3118808BD8B6900221A604FF004
:10354000FF338361FFF7CEFF0023F2E7D1E90032BA
:1035500013605A60F3E70000FFF7C4BF054BD9685A
:103560000875186802681A60536001220275D860F5
:10357000FCF7D0BE284A002030B50C4BDD684B1C50
:1035800087B004460FD02B46094A684600F046F93A
:103590002046FFF7E3FF009B13B1684600F048F9AF
:1035A000A86907B030BDFFF7D9FFF9E7284A002026
:1035B0001D350008044B1A68DB6890689B689842C8
:1035C00094BF002001207047284A0020084B10B506
:1035D0001C68D86822681A60536001222275DC607A
:1035E000FFF78EFF01462046BDE81040FCF792BE73
:1035F000284A002038B5074C074908480123002510
:103600002370656000F028FC0223237085F3118885
:1036100038BD00BF904C0020804B0008284A002095
:1036200008B572B6044B186500F0E2FA00F08EFBA4
:10363000024B03221A70FEE7284A0020904C00201B
:1036400000F02CB98B60022308618B82084670471A
:103650008368A3F1840243F8142C026943F8442CD4
:10366000426943F8402C094A43F8242CC26843F8C5
:10367000182C022203F80C2C002203F80B2C044A0D
:1036800043F8102CA3F12000704700BF2D03000861
:10369000284A002008B5FFF7DBFFBDE80840FFF728
:1036A0005BBF0000024BDB6898610F20FFF756BF3D
:1036B000284A0020302383F31188FFF7F3BF00006E
:1036C00008B50146302383F311880820FFF754FF23
:1036D000002383F3118808BD064BDB6839B14268CB
:1036E00018605A60136043600420FFF745BF4FF035
:1036F000FF307047284A00200368984206D01A68B5
:103700000260506099611846FFF726BF70470000BD
:1037100010B503689C68A2420CD85C688A600B6094
:103720004C602160596099688A1A9A604FF0FF33A3
:10373000836010BD1B68121BECE700000A2938BF2C
:103740000A2170B504460D460A26601900F07EFB7A
:1037500000F06AFB041BA54203D8751C2E460446E4
:10376000F3E70A2E04D9BDE87040012000F0B4BB95
:1037700070BD0000F8B5144B0D46D96103F110017E
:1037800041600A2A1969826038BF0A2201604860D4
:103790001861A818144600F04BFB0A2700F044FB00
:1037A000431BA342064606D37C1C281900F04EFB9F
:1037B00027463546F2E70A2F04D9BDE8F840012034
:1037C00000F08ABBF8BD00BF284A0020F8B50646C5
:1037D0000D4600F029FB0F4A134653F8107F9F4215
:1037E00006D12A4601463046BDE8F840FFF7C2BF81
:1037F000D169BB68441A2C1928BF2C46A34202D9B0
:103800002946FFF79BFF224631460348BDE8F840B2
:10381000FFF77EBF284A0020384A002010B4C0E9D4
:10382000032300235DF8044B4361FFF7CFBF000083
:1038300010B5194C236998420DD0D0E90032816847
:1038400013605A609A680A449A60002303604FF03C
:10385000FF33A36110BD2346026843F8102F536065
:103860000022026022699A4203D1BDE8104000F0B4
:10387000E7BA936881680B44936000F0D5FA226937
:10388000E1699268441AA242E4D91144BDE81040AB
:10389000091AFFF753BF00BF284A00202DE9F0475F
:1038A000DFF8BC8008F110072C4ED8F8105000F05B
:1038B000BBFAD8F81C40AA68031B9A423ED81444AD
:1038C000D5E900324FF00009C8F81C4013605A6077
:1038D000C5F80090D8F81030B34201D100F0B0FA2A
:1038E00089F31188D5E9033128469847302383F3BB
:1038F00011886B69002BD8D000F096FA6A69A0EBAA
:1039000004094A4582460DD2022000F0E5FA002261
:10391000D8F81030B34208D151462846BDE8F047E8
:10392000FFF728BF121A2244F2E712EB090938BF49
:103930004A4629463846FFF7EBFEB5E7D8F810307F
:10394000B34208D01444211AC8F81C00A960BDE88D
:10395000F047FFF7F3BEBDE8F08700BF384A00200C
:10396000284A002038B500F05FFA054AD2E9084538
:10397000031B181945F10001C2E9080138BD00BF59
:10398000284A002000207047FEE700007047000032
:103990004FF0FF3070470000BFF34F8F024AD368EB
:1039A000DB03FCD4704700BF003C024008B5094B64
:1039B0001B7873B9FFF7F0FF074B1A69002ABFBFE6
:1039C000064A5A6002F188325A601A6822F480620C
:1039D0001A6008BD984C0020003C02402301674556
:1039E00008B50B4B1B7893B9FFF7D6FF094B1A6943
:1039F00042F000421A611A6842F480521A601A6852
:103A000022F480521A601A6842F480621A6008BD7B
:103A1000984C0020003C02400728F0B516D80C4C0A
:103A20000C4923787BB90C4D0E4608234FF00062F9
:103A300055F8047B46F8042B013B13F0FF033A448E
:103A4000F6D10123237051F82000F0BD0020FCE7DF
:103A5000BC4C00209C4C00208C4B0008014B53F8C0
:103A6000200070478C4B000808207047072810B5CD
:103A7000044601D9002010BDFFF7CEFF064B53F8D6
:103A800024301844C21A0BB90120F4E7126801323D
:103A9000F0D1043BF6E700BF8C4B0008072810B5B7
:103AA000044621D8FFF778FFFFF780FF0F4AF32382
:103AB000D360C300DBB243F4007343F0020313612D
:103AC000136943F480331361FFF766FFFFF7A4FF28
:103AD000074B53F8241000F035F9FFF781FF20461B
:103AE000BDE81040FFF7C2BF002010BD003C0240FF
:103AF0008C4B0008F8B512F00103144642D185182A
:103B00002E4A954257D82E4B1B6813F0010352D012
:103B10002C4DFFF74BFFF323EB60FFF73DFF40F227
:103B20000127032C15D824F001046618254C401AEF
:103B300040F20117B142236900EB010524D123F0C3
:103B400001032361FFF74CFF0120F8BD043C043062
:103B5000E7E78307E7D12B6923F440732B612B69D7
:103B60003B432B6151F8046B0660BFF34F8FFFF7A7
:103B700013FF03689E42E9D02B6923F001032B61F8
:103B8000FFF72EFF0020E0E723F440732361236951
:103B90003B4323610B882B80BFF34F8FFFF7FCFE65
:103BA0002D8831F8023BADB2AB42C3D0236923F07C
:103BB00001032361E4E71846C7E700BF00000808D7
:103BC00000380240003C0240084908B50B7828B193
:103BD0001BB9FFF7EBFE01230B7008BD002BFCD0D7
:103BE000BDE808400870FFF7FBBE00BF984C0020FE
:103BF0000149024800F0A8B800FF030000010020BE
:103C00000846114600F0CCBE012000F0C9BE0000FD
:103C1000084600F0E3BE000038B5EFF311859DB90A
:103C2000EFF30584C4F30804302334B183F311881F
:103C3000FFF798FE85F3118838BD83F31188FFF7ED
:103C400091FE84F3118838BDBDE83840FFF78ABE85
:103C500038B5FFF7E1FF114C114AC00840EA417046
:103C6000A0FB025EC908A0FB040C1CEB050CA1FB29
:103C700004404FF000035B41A1FB02121CEB040C5B
:103C800043EB000011EB0E0142F10002411842F13A
:103C90000000090941EA007038BD00BFCFF753E3C7
:103CA000A59BC42010B50244064BD2B2904200D16D
:103CB00010BD441C00B253F8200041F8040BE0B2E0
:103CC000F4E700BF502800400F4B30B51C6F2404B0
:103CD00007D41C6F44F400741C671C6F44F4004448
:103CE0001C670A4C236843F4807323600244084B2A
:103CF000D2B2904200D130BD441C00B251F8045BF6
:103D000043F82050E0B2F4E7003802400070004071
:103D10005028004007B5012201A90020FFF7C2FF8B
:103D2000019803B05DF804FB13B50446FFF7F2FFFA
:103D3000A04205D0012201A900200194FFF7C4FF91
:103D400002B010BD704700007047000070470000CF
:103D5000074B45F255521A6002225A6040F6FF7234
:103D60009A604CF6CC421A60024B01221A707047DE
:103D700000300040C44C0020034B1B781BB1034BA8
:103D80004AF6AA221A607047C44C00200030004056
:103D9000034B1A681AB9034AD2F874281A6070479C
:103DA000C04C002000300240024B4FF08072C3F83C
:103DB000742870470030024008B5FFF7E9FF024B56
:103DC0001868C0F3407008BDC04C002008B5FFF76C
:103DD000DFFF024B1868C0F3007008BDC04C002024
:103DE00070470000FEE700000A4B0B480B4A904268
:103DF0000BD30B4BDA1C121AC11E22F003028B42AA
:103E000038BF00220021FDF769B953F8041B40F8C0
:103E1000041BECE7404D00082852002028520020E7
:103E20002852002000F0CAB84FF08043586A70470B
:103E30004FF08043002258631A610222DA60704713
:103E40004FF080430022DA60704700004FF080435B
:103E500058637047FEE7000070B51B4B01630025F7
:103E6000044686B0586085620E46FFF7D7FA04F123
:103E70001003C4E904334FF0FF33C4E90635C4E945
:103E80000044A560E562FFF7CFFF2B460246C4E978
:103E9000082304F134010D4A256580232046FFF7ED
:103EA000D1FB0123E0600A4A037500927268019217
:103EB000B268CDE90223074B6846CDE90435FFF728
:103EC000E9FB06B070BD00BF904C0020AC4B000871
:103ED000B14B0008553E0008024AD36A1843D0622D
:103EE000704700BF284A00204B6843608B6883609E
:103EF000CB68C3600B6943614B6903628B694362A2
:103F00000B6803607047000008B5234B23481A690B
:103F100042F0FF021A611A6922F0FF021A611A695F
:103F20001A6B42F0FF021A631A6D42F0FF021A6523
:103F30001B4A1B6D1146FFF7D7FF02F11C0100F56C
:103F40008060FFF7D1FF02F1380100F58060FFF7D4
:103F5000CBFF02F1540100F58060FFF7C5FF02F1CD
:103F6000700100F58060FFF7BFFF02F18C0100F5E2
:103F70008060FFF7B9FF02F1A80100F58060FFF74C
:103F8000B3FF02F1C40100F58060FFF7ADFFBDE8AB
:103F9000084000F08DB800BF003802400000024029
:103FA000B84B000808B500F027FAFFF723FBBDE87F
:103FB0000840FFF7EDBE0000704700000F4B1A6C81
:103FC00042F001021A641A6E42F001021A660C4AAB
:103FD0001B6E936843F0010393604FF080433122DE
:103FE0009A624FF0FF32DA6200229A615A63DA6015
:103FF0005A6001225A611A60704700BF00380240BF
:10400000002004E04FF0804208B51169D3680B40EE
:10401000D9B2C9439B07116107D5302383F31188B7
:10402000FFF70EFB002383F3118808BD1E4B1A69AE
:1040300062F0FF021A611A69D2B21A614FF0FF30C2
:104040001A695A69586100215A6959615A691A6A8C
:1040500062F080521A621A6A02F080521A621A6A78
:104060005A6A58625A6A59625A6A1A6C42F0805205
:104070001A641A6E42F080521A661A6E0B4A106861
:1040800040F480701060186F00F44070B0F5007F4D
:104090001EBF4FF4803018671967536823F400730C
:1040A000536000F07DB900BF00380240007000404E
:1040B0003B4B3C4A1A643C4A4FF4404111601A6839
:1040C00042F001021A601A689007FCD59A6822F043
:1040D00003029A60324B9A6812F00C02FBD1196805
:1040E00001F0F90119609A601A6842F480321A608E
:1040F0001A689103FCD55A6F42F001025A67284BA7
:104100005A6F9207FCD5294A5A601A6842F08072A9
:104110001A60254A53685804FCD5214B1A6891014E
:10412000FCD5234AC3F884201A6842F080621A60E2
:104130001A681201FCD51F4A9A600322C3F88C202A
:104140004FF00062C3F894201B4B1A681B4B9A4235
:104150001B4B21D11B4A11681B4A91421CD140F2D2
:1041600003121A60164A136803F00F03032BFAD1E7
:104170000B4B9A6842F002029A609A6802F00C02B5
:10418000082AFAD15A6C42F480425A645A6E42F4B8
:1041900080425A665B6E704740F20372E1E700BFEF
:1041A000003802400004001000700040081940026E
:1041B0001030002400948838002004E011640020AE
:1041C000003C024000ED00E041C20F41074A08B543
:1041D000536903F00103536123B1054A13680BB11E
:1041E00050689847BDE80840FFF73CB9003C0140E3
:1041F000C84C0020074A08B5536903F00203536115
:1042000023B1054A93680BB1D0689847BDE80840D0
:10421000FFF728B9003C0140C84C0020074A08B508
:10422000536903F00403536123B1054A13690BB1C9
:1042300050699847BDE80840FFF714B9003C0140B9
:10424000C84C0020074A08B5536903F008035361BE
:1042500023B1054A93690BB1D0699847BDE808407E
:10426000FFF700B9003C0140C84C0020074A08B5E0
:10427000536903F01003536123B1054A136A0BB16C
:10428000506A9847BDE80840FFF7ECB8003C014091
:10429000C84C0020164B10B55C6904F478725A6162
:1042A000A30604D5134A936A0BB1D06A98476006F7
:1042B00004D5104A136B0BB1506B9847210604D5F7
:1042C0000C4A936B0BB1D06B9847E20504D5094AB1
:1042D000136C0BB1506C9847A30504D5054A936C39
:1042E0000BB1D06C9847BDE81040FFF7BBB800BFDA
:1042F000003C0140C84C0020194B10B55C6904F427
:104300007C425A61620504D5164A136D0BB1506D9B
:104310009847230504D5134A936D0BB1D06D984788
:10432000E00404D50F4A136E0BB1506E9847A104F8
:1043300004D50C4A936E0BB1D06E9847620404D535
:10434000084A136F0BB1506F9847230404D5054AF0
:10435000936F0BB1D06F9847BDE81040FFF782B85C
:10436000003C0140C84C002008B5034800F010F99B
:10437000BDE80840FFF776B8484D002008B503486F
:1043800000F006F9BDE80840FFF76CB8B44F002014
:1043900008B5FFF737FEBDE80840FFF763B8000037
:1043A000062108B50846FFF787F806210720FFF722
:1043B00083F806210820FFF77FF806210920FFF780
:1043C0007BF806210A20FFF777F806211720FFF770
:1043D00073F806212820FFF76FF807211C20FFF74C
:1043E0006BF80C212520FFF767F8BDE808400C2189
:1043F0002620FFF761B8000008B5FFF717FE00F0B0
:104400007BF800F03DF8FFF7D7FDBDE80840FFF767
:1044100009BD0000026843681143016003B11847F9
:1044200070470000143000F0DFB900004FF0FF3398
:10443000143000F0D9B90000383000F055BA00004F
:104440004FF0FF33383000F04FBA0000143000F066
:10445000A5B900004FF0FF31143000F09FB9000003
:10446000383000F0FFB900004FF0FF32383000F074
:10447000F9B90000012914BF6FF013000020704744
:1044800000F060B837B515460E4A0260002242605F
:10449000C0E902220122044602740B46009000F19A
:1044A0005C014FF48072143000F04EF900942B46FA
:1044B0004FF4807204F5AE7104F1380000F0C6F9D3
:1044C00003B030BD984C000838B5C36904460D46AA
:1044D0001BB904210844FFF79DFF294604F114008D
:1044E00000F040F9002806DA201D4FF40061BDE815
:1044F0003840FFF78FBF38BD0023054A1946013306
:10450000102BC2E9001102F10802F8D1704700BF78
:10451000C84C0020026843681143016003B118478A
:1045200070470000024AD36843F0C003D36070476D
:1045300000100140024AD36843F0C003D3607047C3
:104540000044004010B50A4C0A4A20460021FFF7FB
:1045500099FF094B094AC4E99723094C094A0021EC
:104560002046FFF78FFF0849084BC4E9971310BD99
:10457000484D00202545000880F0FA020010014057
:10458000B44F0020354500080044004040787D01CC
:104590002DE9F041D0F85C62F7683368DA0504462B
:1045A0009DB20DD5302383F311884FF48061043020
:1045B000FFF7B0FF6FF480733360002383F311883B
:1045C000302383F3118804F1040815F02F033AD146
:1045D00083F31188380615D5290613D5302383F3C4
:1045E000118804F1380000F065F900284EDA08213E
:1045F000201DFFF78FFF4FF67F733B40F3600023D2
:1046000083F311887A0616D56B0614D5302383F30D
:104610001188D4E913239A420AD1236C43B127F0BD
:1046200040073F041021201D3F0CFFF773FFF76088
:10463000002383F31188D4F86822D36843B3BDE81C
:10464000F041106918472B0714D015F0080F0CBF64
:1046500000214FF48071E80748BF41F02001AA070C
:1046600048BF41F040016B0748BF41F08001404620
:10467000FFF750FFAD06736805D594F86412204625
:104680001940FFF721FF3568ADB29EE77060B6E7CD
:10469000BDE8F081F8B5154682680669AA420B4666
:1046A000816938BF8568761AB54204460BD2184630
:1046B0002A46FCF701FDA3692B44A361A3685B1B99
:1046C000A3602846F8BD0CD918463246FCF7F4FC26
:1046D000AF1BE1683A463044FCF7EEFCE3683B442C
:1046E000EBE718462A46FCF7E7FCE368E5E700003D
:1046F00083689342F7B51546044638BF8568D0E90C
:104700000460361AB5420BD22A46FCF7D5FC636921
:104710002B446361A36828465B1BA36003B0F0BD14
:104720000DD932460191FCF7C7FC0199E068AF1B37
:104730003A463144FCF7C0FCE3683B44E9E72A46CB
:10474000FCF7BAFCE368E4E710B50A440024C3614F
:10475000029B8460C0E90000C0E90511C1600261EC
:10476000036210BD08B5D0E90532934201D18268D9
:1047700082B98268013282605A1C42611970D0E9A4
:1047800004329A4224BFC36843610021FEF7B4FF9C
:10479000002008BD4FF0FF30FBE7000070B530236C
:1047A00004460E4683F31188A568A5B1A368A269E3
:1047B000013BA360531CA36115782269934224BF77
:1047C000E368A361E3690BB120469847002383F3B4
:1047D0001188284607E031462046FEF77DFF002875
:1047E000E2DA85F3118870BD2DE9F74F04460E46D5
:1047F00017469846D0F81C904FF0300A8AF311887B
:104800004FF0000B154665B12A4631462046FFF7AA
:1048100041FF034660B941462046FEF75DFF002890
:10482000F1D0002383F31188781B03B0BDE8F08F2B
:10483000B9F1000F03D001902046C847019B8BF3CC
:104840001188ED1A1E448AF31188DCE7C0E90511CE
:10485000C160C3611144009B8260C0E90000016136
:1048600003627047F8B504460D461646302383F3BD
:104870001188A768A7B1A368013BA36063695A1CAC
:1048800062611D70D4E904329A4224BFE368636117
:10489000E3690BB120469847002080F3118807E0B8
:1048A00031462046FEF718FF0028E2DA87F3118828
:1048B000F8BD0000D0E905239A4210B501D1826805
:1048C0007AB98268013282605A1C82611C7803695D
:1048D0009A4224BFC36883610021FEF70DFF204682
:1048E00010BD4FF0FF30FBE72DE9F74F04460E46B1
:1048F00017469846D0F81C904FF0300A8AF311887A
:104900004FF0000B154665B12A4631462046FFF7A9
:10491000EFFE034660B941462046FEF7DDFE002863
:10492000F1D0002383F31188781B03B0BDE8F08F2A
:10493000B9F1000F03D001902046C847019B8BF3CB
:104940001188ED1A1E448AF31188DCE70B460146F4
:10495000184600F02DB8000000F040B8012838BF1C
:10496000012010B50446204600F030F830B900F0C0
:1049700007F808B900F00CF88047F4E710BD000014
:10498000024B1868BFF35B8F704700BF20520020B6
:1049900008B5062000F084F80120FEF7F5FF0000BE
:1049A000024B0A4601461868FFF72AB91C2300206B
:1049B00010B5054C13462CB10A4601460220AFF350
:1049C000008010BD2046FCE700000000024B0146BD
:1049D0001868FFF719B900BF1C230020024B0146DD
:1049E0001868FFF715B900BF1C23002010B5013966
:1049F0000244904201D1002005E0037811F8014FF4
:104A0000A34201D0181B10BD0130F2E72DE9F0419F
:104A1000A3B1C91A17780144044603F1FF3C8C4244
:104A2000204601D9002009E00578BD4204F10104C7
:104A3000F5D10CEB0405D618A54201D1BDE8F081F3
:104A400015F8018D16F801EDF045F5D0E7E7000007
:104A50001F2938B504460D4604D9162303604FF0CC
:104A6000FF3038BD426C12B152F821304BB92046AC
:104A700000F030F82A4601462046BDE8384000F0F4
:104A800017B8012B0AD0591C03D11623036001204B
:104A9000E7E7002442F82540284698470020E0E751
:104AA000024B01461868FFF7D3BF00BF1C2300204C
:104AB00038B5074D00230446084611462B60FEF723
:104AC00067FF431C02D12B6803B1236038BD00BFD0
:104AD00024520020FEF756BF034611F8012B03F8BD
:104AE000012B002AF9D170476F72672E61726475CD
:104AF00070696C6F742E435541565F4750530000E8
:104B000040A2E4F1646891060041A3E5F265699270
:104B1000070000004261642043414E4966616365BD
:104B200020696E6465782E0080000000008000001F
:104B300000008000000000000000000031190008A3
:104B400051210008AD200008711900087D190008E6
:104B50007D1B00084119000851190008451900087B
:104B60004D19000849190008A11A00085519000834
:104B70002124000865190008751A00086330000038
:104B80007C4B0008804A0020904C00200040000030
:104B90000040000000400000004000000000010054
:104BA0000000020000000200000002006D61696E5A
:104BB0000069646C65000000A0011028000000007E
:104BC000AAAAAAAA50011024FFFF00000077000043
:104BD0000000000000A40A0100000000AAA6AAAA82
:104BE00080500000DFEF0000000000778800000028
:104BF0000000000000000000AAAAAAAA000000000D
:104C0000FFFF0000000000000000000000000000A6
:104C100000000000AAAAAAAA00000000FFFF0000EE
:104C20000000000000000000000000000000000084
:104C3000AAAAAAAA00000000FFFF000000000000CE
:104C4000000000000000000000000000AAAAAAAABC
:104C500000000000FFFF0000000000000000000056
:104C60000000000000000000AAAAAAAA000000009C
:104C7000FFFF000000000000000000000000000036
:104C8000000000000A000000000000000300000017
:104C90000000000000000000000000004144000887
:104CA0002D44000869440008554400086144000888
:104CB0004D440008394400082544000875440008A4
:104CC000E9030000000000000000070000000000F1
:104CD00040420F00FE2A0100D204000020230020E1
:104CE00000000000000000000000000000000000C4
:104CF00000000000000000000000000000000000B4
:104D000000000000000000000000000000000000A3
:104D10000000000000000000000000000000000093
:104D20000000000000000000000000000000000083
:104D30000000000000000000000000000000000073
:00000001FF
